:020000040800F2
:10500000501A0020D550000871820008817A0008EB
:105010000000000000000000000000000000000090
:10502000000000000000000000000000D58F000814
:105030000000000000000000B1880008E9900008AE
:10504000E7500008E7500008E7500008E750000864
:10505000E7500008295B0008E7500008E750000807
:1050600000000000E7500008515A0008E75000080F
:10507000E7500008ED7E000800000000E75000083F
:1050800000000000E75000080000000000000000E1
:10509000E750000800000000E7500008E750000853
:1050A000E7500008E7500008E7500008799800082A
:1050B000E7500008E7500008000000000000000072
:1050C0000348854600F060FC004800478DA60008B4
:1050D000501A00200448804704480047FEE7FEE7D6
:1050E000FEE7FEE7FEE7FEE785910008C1500008F5
:1050F00030B50B46014600202022012409E00D4670
:10510000D5409D4205D31D469540491B25469540F7
:1051100040191546521E002DF1DC30BDF0B51FB40C
:105120000646002082B005464024019100901BE015
:10513000019922460F46304600F04EFB049A059B2B
:10514000801A994110D310461946224600F034FBCC
:10515000361A8F410197224601200021009F00F05E
:105160002BFB38184D4100902046641E0028DFDCE0
:10517000019B00982946324607B0F0BD03460B4319
:105180009B0703D009E008C9121F08C0042AFAD2FD
:1051900003E00B780370401C491C521EF9D2704783
:1051A000D2B201E00270401C491EFBD270470022BF
:1051B000F6E710B513460A4604461946FFF7F0FF16
:1051C000204610BD30B504460020034600E05B1CBD
:1051D000934203D2E05CCD5C401BF8D030BDF8B503
:1051E00002464A40D40F42004B0052085B089A42E4
:1051F00002D20246084611464A0023D0C30D4A0097
:10520000DDB2120EAD1A202D35DA49020126490A07
:10521000F6058A19002C00D0524220214F1B11465E
:10522000B9402A411018C20D9A4221D0002C17D043
:10523000012D08DCDA05801AD20F8019D207DBB203
:1052400000F0F6FAF8BDDA05801A012340001B06CB
:10525000C01880185A428018CA0F1043490007E04E
:105260004908C2071143DA05801A801940088018DE
:1052700000F0D6FAF8BD61000122511A001BF7E7D1
:105280000122D2075140AAE70122D2075040A6E7E7
:1052900070B502464A40D50F40004A00ED0740086D
:1052A0005208002814D0002A12D0C40DD30D410298
:1052B0000120C0055202490A520AE41A09181218BC
:1052C0007D34914201D3641C00E04900002C01DAD6
:1052D000002070BD0023914201D3891A0343400886
:1052E00049000028F7D100290AD0914202D10121BA
:1052F000C90705E0914201D2012101E00121C94322
:10530000E005C018401900F08BFA70BDF0B50746F3
:105310000846584087B0C00F049048000E46590018
:1053200040084908BC1A884105D2384631461E4615
:1053300017460B4602465800400810434CD0300D2B
:10534000039040055900400D490D0590401A029008
:10535000402872DA18030121000B09050843019067
:1053600004980092002805D00199524200208841FB
:1053700000920190029840210A1A0199009800F0C9
:105380001BFA05460C466B4607CB00F036FAC019EF
:105390007141039A0E0D0023D71756401A467A40E2
:1053A000164344D0049A002A2DD0029A012A039A67
:1053B00015DC1205C01A914101263605001C714109
:1053C000D20F059ED2070093019202962A462346E9
:1053D00000F074FA07B0F0BD38463146FAE716051A
:1053E000224A0F46B218C01AB74101210905001C14
:1053F0004F4100187F41114618187941E20F1043C0
:105400006D19644113E0E2076D0815436408C20793
:105410001443039A01261205C01A91413605001C57
:105420007141CE07400830434908C01851412A460F
:10543000234600F036FACDE7FFE70498012240004A
:10544000C117121A00238B4104983146C417381A29
:10545000A141EEE730B40124E407634030BC55E7D6
:1054600030B40124E407614030BC4FE70000E0FFA6
:10547000F0B51FB488B00B990998002448400999E9
:10548000C00F490049080991C0070B9900904900D5
:1054900049080B9109990898A64608431CD00B9916
:1054A0000A98084318D0099801244000420D48008A
:1054B000410D099824050003000B204309900B9827
:1054C0000003000B20430B9050181C494018002289
:1054D00001901446104605E0002001460DB0F0BDD5
:1054E000032801DA034600E003239C46C11A0AAEF2
:1054F0000AE05F0008ADED5B4F00F75B7D430027DE
:10550000AA187C41491C5B1E6145F2DD410004ABD9
:105510005A522104120C0A43240C401C0828DFDBD9
:10552000019802900099704601910090059B049AA1
:105530000799069800F0C2F9D0E700000DFCFFFFC4
:10554000F0B50C465C4085B0E40FE40703944C00D2
:1055500000266408590094464908024602962243F0
:1055600021D062460A431ED06200570D4A000E0346
:105570002303550D012402462C492405781B1B0BDF
:10558000360B401823432643614600901C46501AB0
:10559000B44103D30098401C009002E09218009898
:1055A0005B41002803DA0020014605B0F0BD002071
:1055B000012109050746864611E064461D46141B75
:1055C000B54106D36546521BB341744607430C43AD
:1055D000A646CD0740084908284392185B41054676
:1055E0000D43EAD11046184313D060461946504087
:1055F0007140084306D06046101AB34106D201221A
:10560000002306E000220123DB0702E00122D2434F
:105610005310009874460105381C6141029C039D9B
:105620000019694100F03DF9BFE70000FD030000EB
:10563000C217C10F504010B54018CA079623002169
:1056400000F0F6F810BD10B500229623114600F0C8
:10565000EFF810BD0EB5C217C10F5040CA07401871
:105660000021054B0293019200910A460B4600F07F
:1056700025F903B000BD0000330400000EB5054954
:105680000291002100910A460B46019100F016F9A3
:1056900003B000BD33040000410040020122400A73
:1056A000D205090E80187F2901DA0020704796295B
:1056B00003DC9622511AC8407047963988407047DB
:1056C00070B5CD0F4A0009030123090B1B051943CF
:1056D0000B4BED070024520D9A4201DA002070BDF9
:1056E000074B34339A4203DC9A1A00F075F802E053
:1056F0000449511888402C43F1D0404270BD00004D
:10570000FF030000CDFBFFFF4A0009030123090B43
:105710001B051943094B10B5520D9A4201DA0020BE
:1057200010BD064B34339A4203DC9A1A00F054F849
:1057300010BD03495118884010BD0000FF03000050
:10574000CDFBFFFFC20FD207400040080BD0C10DB8
:105750000723DB01C91840020905400A1143C208AA
:10576000400711437047002001467047CB0FDB070D
:10577000490010B5490802460A4307D00A0D07241C
:105780000903E401090B121B002A01DC002010BDF3
:10579000C900440F0C43C100E018D205801800F086
:1057A0003FF810BD0122D207002800DB101A0029A3
:1057B00000DB511A8142704710B5202A04DB0146F4
:1057C000203A9140002010BD914020239C1A0346AE
:1057D000E3401943904010BD10B5202A04DB084671
:1057E000203AD040002110BD0B46D340D0402024A9
:1057F000A21A91400843194610BD10B5202A06DBB5
:10580000CB170846203A1041C1170B4306E00B4660
:105810001341D0402024A21A91400843194610BDDC
:10582000002904DA401C490001D1400840007047BB
:1058300070B40024050C05D11024000402D1002905
:1058400021D01124050E01D100020834050F01D129
:105850000001241D850F01D18000A41C002801DB5C
:105860004000641C002908D020252E1B0D46F54061
:10587000A14000D001212943084301061B1B000A57
:10588000DB1D02D5002070BC7047DB05181880189E
:105890000029F8DA401C4900F5D170BC40084000EE
:1058A000704710B5002B08DA0024401C61419218A3
:1058B0005B411A4301D14008400010BDF0B51FB450
:1058C00082B005460C0003D0084604F095F802E0CB
:1058D00004F092F820300246009021462846FFF757
:1058E0006BFF049B059A04460F4618431143084377
:1058F00014D0184610431BD0009840210A1A1846AD
:105900000599FFF769FF05460E46009A0599049828
:10591000FFF752FF084305D0012004E02046394636
:1059200007B0F0BD0020C11705430E432C43374399
:1059300000990E986305401A7905E40A00220C4389
:10594000FD0A0A3002D500200146E9E701051019D9
:1059500069410C9C0D9D00196941FFF7A2FFDFE72B
:1059600010B5002904DB0124E40740428C412146A4
:10597000002B04DB1C460123DB075242A341994262
:1059800000D1904210BD0000064C0125064E05E0F6
:10599000E36807CC2B430C3C98471034B442F7D350
:1059A000FFF792FBECA900080CAA000838B50446E2
:1059B000064805490068FFF79BFB604300E0401E76
:1059C00000900028FBD138BD40420F0004010020A8
:1059D000F8B50446006881688907890F012902D15A
:1059E0000168C90722D18168114A1026114001259A
:1059F00000290ED18168294381600120FFF7D6FF7D
:105A000000F0AAFF07460CE000F0A6FFC01B0A2822
:105A100007D9606D30436065A06D2843A065012003
:105A2000F8BD20680068C043C007EDD10020F8BD74
:105A30001700008010B500231A4603E0845CE318C9
:105A40009BB2521C8A42F9D3D84380B210BD0000E9
:105A500010B5034800F040FD024800F03DFD10BDC8
:105A6000F0150020A815002030B5446C1C252C40F2
:105A70000125A540046C6560046863608368102B91
:105A8000036803D099600068C26030BD9A60006806
:105A9000C16030BD1449012048720A4602205E32BE
:105AA000507203203C3A507204200E3A50720F4854
:105AB0000D4B0078087022310870203108770C49AE
:105AC0005A1C0878587149789971233318715971A3
:105AD000203318775977107551751A461E32107594
:105AE000517510765176704738110020C70000209C
:105AF000E400002010B503F045FA202003F0EAFA94
:105B0000012004F029FB002003F0E4FA044804F02B
:105B1000C7F9044804F06AFC002004F09FFC10BDA3
:105B2000B00000208380000070B50520012100072F
:105B300000F002FF00240D4D002800D02C6002214F
:105B40000B4800F0F9FE002808D10A482C600088B4
:105B50000A2148430849088003F0A0FE012000F014
:105B600023FE022000F020FE70BD0000FC0000209B
:105B700000040050D4000020E00000207047000026
:105B800010B5084900224A6107494B684C15234368
:105B90004B604B68082423434B60C009C00102607E
:105BA00010BD000038160020002002407FB50025FF
:105BB0000C460646039500F0C7FDE009029003A9D4
:105BC00001960095684600F057FD002804D000F0CB
:105BD0008FFD002004B070BD00F08AFD0120F9E7C0
:105BE00010B5002302E0C45CCC545B1C9342FAD392
:105BF00010BD000010B5214A00219069C30520485E
:105C000004D54169022319434161911593699B05AC
:105C100005D5436901242343436163021943936912
:105C20005B0505D54369082423434361E301194318
:105C300093691B0505D5436904242343436163022B
:105C4000194393699B0405D5436910242343436199
:105C50006302194393699B0304D5446920231C43C1
:105C6000446119439369DB0305D543694024234309
:105C70004361A0020143916110BD00000020024079
:105C80003816002070B5054600F066FE0646184C32
:105C90000AE0681C08D0002D04D000F05DFE801BD7
:105CA000A84201D9032070BDA069C007F1D1A06945
:105CB000800701D50220A061A069C00511D4A069A8
:105CC00080050ED4A06940050BD4A069000508D456
:105CD000A069800405D4A069800302D4A069C00330
:105CE00003D5FFF787FF012070BD002070BD0000C5
:105CF00000200240F8B51746002605460C4600F085
:105D000023FD09E029460220226800F0FFFC00285C
:105D100004D1241D2D1D361DBE42F3D300F0E8FC36
:105D2000BE4201D20020F8BD0120F8BD10B50849DF
:105D300002460020054B497905E044001C5B944273
:105D400003D0401CC0B28842F7D310BD60120020BF
:105D50004800002010B500F0F4FD10BD10B5094852
:105D600000F0A0FF80B2FFF789FC074A074BFFF75E
:105D70007FFB0022064BFFF7E3FBFFF7C5FC80B279
:105D800010BD0000A0140020F853E3A59B843E4002
:105D900000408F40F8B540493E488A7F0275C97F70
:105DA00041753E490A78027649784176394905209D
:105DB000133148720A2004F009FB7D20C00004F072
:105DC0001FFB3449002213310C2004F0E9FB0021B1
:105DD0000C2004F0F7FB022004F048FB304D2E4C61
:105DE00000210F2004F072FA28422063F8D0206BC3
:105DF000411C40D02B4E2C4F40043ED58122D20175
:105E000000210F2004F0A1FB0021102004F05EFA15
:105E100041062048490E0022633004F08DFA1D4DE2
:105E20006335687A052825D102221C49681DFFF7D1
:105E3000C9F900281ED1A87C607117480422691C8A
:105E40004430FFF79BF9606C00F034F8A083607970
:105E500029464200133108465130FFF78FF91348A5
:105E600031888088FFF744F9388841431048018021
:105E700003202070F8BD02F01FFAA08B3188054680
:105E8000FFF736F93888414309486D1E0180A58324
:105E9000F8BD00009911002048000020E400002017
:105EA00000D02724D0000020CE000020380D002094
:105EB000CC00002010B504460E4800F0F3FE0E4959
:105EC000C006C00E098805E02246C240D2070FD0A6
:105ED000401CC0B28842F7D3012005E02246C240F0
:105EE000D20705D0401CC0B28842F7D3491EC8B2C1
:105EF00010BD0000A0140020D000002010B50848FC
:105F000000F096FA0A21064800F032FA044800F040
:105F10001DF9800503D5024800F01AF980B210BDC2
:105F200044140020F8B52F4D00220121284600F02E
:105F30000CFDFFF7E3FFFFF786FB2B4E3146FFF723
:105F4000A7F92A4C0122A0601146284600F0FDFC6A
:105F50002749A068002588423EDB2078254F00288D
:105F600015D02570FFF7CAFFFFF76DFB3146FFF72D
:105F70008FF9A060FFF7E6FB00223B46FFF76AFAC5
:105F800000221D4BFFF774FAFFF7F0FB6060A0687A
:105F9000FFF7D8FB00223B46FFF75CFA174A184B85
:105FA000FFF766FA06460F466068FFF7CBFB134A19
:105FB000144B5242FFF75CFA32463B46FFF7A6F914
:105FC000FFF7D4FB10496060884201DD616004E0A6
:105FD000FF21C905C84200D365606068FFF75CFB1C
:105FE000C0B2F8BD0004005000401B442400002053
:105FF0000000604000000C4000E064403333333365
:1060000033B33040CCCCEC3F0000C842F8B5054675
:1060100004464035287C0026012808D00120287439
:10602000206881688907890F01290ED101E00220CB
:10603000F8BD0168C90708D0606D2021084360657C
:106040000126002028743046F8BD616DFF22013220
:106050009143022211436165C1688907890F00914C
:10606000C16889088900C16020688168920711436E
:10607000816000F071FC07460EE000F06DFCC01B73
:106080000A2809D9606D0221884310210843606500
:10609000002028740120F8BD206880680028ECDB0F
:1060A0002068C168009A1143C160606D800880005B
:1060B000401C6065C5E70000F8B506460D46403651
:1060C000317C01290DD00121317401688A685207A1
:1060D00009D5416D20221143416500203074012013
:1060E000F8BD0220F8BD174B6A68D80547109A42E0
:1060F000154C8A6A2B6812D05B035B0B1A438A62C9
:106100002968490305D5A1680143A1600A20FFF76A
:106110004DFC2868800312D5A06838430EE05B036D
:106120005B0B9A438A622968490302D5A1688143BF
:10613000A1602868800302D5A068B843A060002051
:106140003074F8BD0110000000270140406D704719
:106150000068006C7047000070B5040006D0606DE8
:10616000264600254036002802D006E0012070BDFA
:10617000A5653574204600F0D3F8606DC00603D4E1
:1061800021688868400705D5606D10210843606567
:106190003574EBE7606DFF22013290430222104319
:1061A000606588688207920F5B48012A02D10A68FD
:1061B000D2072BD1032362689B079A4205D05B422A
:1061C0009A4202D05B009A4209D10A699200920871
:1061D0000A6121680A6963681A430A610CE00A6966
:1061E000920092080A6181680F22920491438160B3
:1061F00081686268114381602168CA6818239A43E4
:10620000CA602168CA68A3681A43CA60816801220B
:106210005206914381608168A28E520611438160CB
:1062200020688168C90004D48168012212071143E3
:1062300081602068C168394A1140C1602069E16805
:10624000022825D000200143204620300278037B1D
:1062500052035B001A431143226B1143A26992035C
:106260001143E269D20311432268D3681943D16014
:10627000616A0A46FF3AC23A05D0A26A114322680F
:10628000D3681943D16042780121012A02D00BE082
:106290000420D8E70078002823D0606D2022104326
:1062A0006065A06D0843A065E06B012820681FD0E1
:1062B0000169C90703D001694908490001612068E3
:1062C0004169C908C900416120684169A26B114355
:1062D0004161A565606D80088000401C60650020FC
:1062E00070BD2068C26801231B041A43C260DBE74B
:1062F0000269FF239B009A43026120680269236CB4
:10630000A66C1A43636C33431A4302612068026926
:106310000A430261D3E70000002701401902FEFF93
:1063200010B586B0044614216846FEF740FF0E49BA
:106330002068884216D10D48416B421511434163D4
:10634000C16A01221143C162C06A694610400590CA
:1063500002200090032001900020029005200007F9
:1063600000F02EFA06B010BD0024014000100240DB
:10637000F8B504464069254640350E4608280BD03E
:106380002068C068C00709D0606D2021084360659F
:10639000002028740120F8BD082700E00C2700F039
:1063A000DBFA009011E0701C0FD0002E05D000F039
:1063B000D3FA0099401AB04207D9606D042108430E
:1063C0006065002028740320F8BD2068006838420A
:1063D000E9D0606D01214902084360652068C16809
:1063E00009058A0F0C21002A1BD12022125D002AE8
:1063F00017D10268120714D5826853070122002BB7
:1064000008DB43688B434360606D1302984310437D
:10641000606506E0606D202318436065A06D104341
:10642000A065A069002801D1206801600020F8BDA6
:1064300070B50446216800208968490721D42546A3
:106440004035297C01291CD001212974E1690129E9
:1064500004D02046FFF7BCFA002811D1616D0A4A2A
:106460001140FF220132114361650021A1652974A9
:1064700022681C21116021688A6804231A438A60FB
:1064800070BD022070BD0000FEF1FFFF70B500245A
:10649000014620314A79022A03D00421C163012434
:1064A00018E0026813680E25AB4313600268136896
:1064B0005B085B001360436C1C22134001221546ED
:1064C0009D40036C5D604A7100220A71816B002956
:1064D00000D08847204670BDF0B4016C0D6801689B
:1064E0000C68466C1C2304221E401746B7402F42FE
:1064F0000ED067070CD50C68A40602D40C68944330
:106500000C60416C19408A40016C4A60016B1AE0D2
:106510000227B74002462F402032002F17D0A7078E
:1065200015D50C68A40605D40C680A25AC430C608C
:1065300001215171446C02211C40036CA14059603F
:1065400000211171C16A002918D0F0BC0847082742
:10655000B7402F4212D0240710D50C680E25AC434B
:106560000C60446C01211C400B46A340046C63602A
:10657000C163517100211171416BE4E7F0BC7047B8
:1065800070B504003CD01F48256814212818FEF778
:10659000AFFD800060641C4820640221204620304A
:1065A0000246417129681948E3680140A06866699C
:1065B0001843236933431843A3691843E369184315
:1065C000236A1843084328600121A0688903884290
:1065D00010D00D488030836A656C1C210D400F2659
:1065E000AE40B3438362656C63680D40816AAB4023
:1065F0000B4383620020E06301215171107170BD73
:10660000012070BDF8FFFDBF000002400F80FFFFBA
:10661000F8B504468C46203001790025012909D0BF
:106620000126067141790027012905D0077102254D
:106630002846F8BD0220F8BD02214171E7632068B9
:10664000016849084900016061462046FFF70CFADD
:10665000206B00282068016801D00E2205E004228A
:1066600091430160206801680A221143016020689B
:10667000016831430160DBE7F8B51A4E0546307C0E
:106680000F46012807D0012030741748FFF7FAFAA7
:10669000010002D021E00220F8BD0020C043386094
:1066A0006C6814E02046FFF76BFA0F48FFF7EAFA30
:1066B00001460E48426808239A43426042684315E7
:1066C0009A434260002901D03C6006E08034A8680B
:1066D0006A68C0018018A042E4D8002030740846DF
:1066E000F8BD00003816002050C300000020024012
:1066F000054841680222114341604168012211436B
:10670000416000207047000000200240F8B50C4CAA
:106710001646207C0F46012808D001202074094825
:10672000FFF7B0FA0025002802D006E00220F8BDED
:1067300065613E600348FFF7A5FA2574F8BD0000C7
:106740003816002050C3000011484168C9070BD01B
:10675000EFF3108172B60F4AC2600F4AC26081F334
:1067600010884168C9070ED1416889070DD5EFF33C
:10677000108172B6094A0261094A026181F31088E8
:106780004068800701D50120704700207047000055
:1067900000200240EFCDAB8905040302BFAE9D8C03
:1067A000161514137047000010B504494A690242D7
:1067B00002D04861FFF7F6FF10BD00000004014061
:1067C000F8B500230124A2E027469F403A4070D04C
:1067D0004D68022D01D0122D14D1DD08AD002D1809
:1067E00000952D6A5E07AC46F50E0F26AE46AE400C
:1067F0006546B543AC460E697546AE4065462E43C8
:10680000009D2E624D68012D05D0022D03D0112D63
:1068100001D0122D16D185680326AC465D00AE4628
:10682000AE406546B543AC46CE687546AE4065465B
:106830002E43866046680D79BE43ED06ED0F9D4000
:106840003543456006685F000325BD40AE46AE4354
:106850000D79B446AE07B60FBE4065462E430660BE
:10686000C6687546AE438D68BD403543C5604D680A
:10687000ED004BD5294D6E6B26436E639E08284D67
:10688000B6007519AC46AD689E07360F0F27B740A6
:10689000BD4305273F07B84201D1002715E0214F2E
:1068A000B84201D1012710E01F4FB84202D10227A0
:1068B0000BE02BE01D4FB84201D1032705E01C4F30
:1068C000B84201D1052700E00627B7402F436546AF
:1068D000AF60184D2E684F689643FF0300D51643EE
:1068E0002E606E684F689643BF0300D516436E60F6
:1068F000AE684F689643FF0200D51643AE60EE685F
:106900004F689643BF0200D51643EE605B1C0A68D1
:106910001546DD4000D057E7F8BD000000100240EA
:10692000000001400004005000080050000C00501E
:10693000001C0050000401400069084000D0012004
:10694000704742694A4042617047002A01D0816124
:10695000704781627047000001480068704700007E
:106960000001002002480168491C016070470000D6
:106970000001002010B5084800240168402211439E
:106980000160204600F00AF8002801D0012401E04F
:1069900000F0B4F9204610BD0020024070B5054655
:1069A00009487D210024C9000068FEF7A1FB00F022
:1069B00049FE002801D0012404E000222946501E8F
:1069C00000F0BCF9204670BD0401002070477047FC
:1069D000F8B52D4C0126A078401CA0702671E08AE5
:1069E000401CE0822948008802F032FB284DE888EC
:1069F000FEF729FE2749FEF74BFC274F3968FEF7C3
:106A0000EEFB386002212548FFF796FF002700289B
:106A100009D027632048224A016822480091914208
:106A200012DD067011E0E888FEF70DFE1949FEF749
:106A30002FFC216BFEF7D3FB1B4920638842E9DB67
:106A40001B491A48C860E5E70770688F401EFEF7CB
:106A5000EFFD0099FEF7A6FE05D86079002802D068
:106A60001448067001E013480770688FFEF7EBFDCD
:106A700009490968FEF796FE04D26079002801D022
:106A800003F088FEF8BD0000C40000206400002070
:106A9000380D002000007A44FC0000200004005063
:106AA000000040404E0000200000A0400400FA0515
:106AB00000ED00E05D000020704770B505000DD0CE
:106AC00002202C462034A073284601F017FA2846ED
:106AD00000F0BEF80020A073607370BD012070BD8F
:106AE0007047704710B5044600680168C943C9077C
:106AF00008D18168C943C90704D1012141602046FA
:106B0000FFF766FF20680168C943890708D48168D8
:106B1000C943890704D4022141602046FFF756FF8C
:106B200020680168C943490708D48168C9434907F7
:106B300004D404214160204600F0DEF8206801689A
:106B4000C943090708D48168C943090704D4082147
:106B500041602046FFF7B0FF20680168C943C906BD
:106B600008D48168C943C90604D410214160204675
:106B7000FFF72DFF20680168C943890608D48168A2
:106B8000C943890604D4202141602046FFF7A9FFAC
:106B900020680168C943490608D48168C943490689
:106BA00004D4402141602046FFF79AFF10BD000049
:106BB000F8B5040005D025462035A87B002802D072
:106BC00006E00120F8BD00206873204600F052F86E
:106BD0000220A8732068C26884466368012B04D031
:106BE0000120A16AC005814201D11E2082431548BF
:106BF0006169814201D0144802401448A6680240ED
:106C000018463043676A266A3E433043A66A3043DB
:106C10001043012B03D00122D205964203D12369F0
:106C2000E2681A431043074A914205D0A269114312
:106C3000E2690243084610436146C8600120A87318
:106C40000020F8BDFFFF00003F1FFFFFF8F119FF14
:106C500010B500680549884207D10548816B490095
:106C6000490881630D2000F055F810BD007C0040FC
:106C70000010024010B50068084988420CD108484D
:106C8000816BC20411438163002201210D2000F0B9
:106C900055F80D2000F048F810BD0000007C0040C1
:106CA000001002400068C0697047000070B50224FF
:106CB000034620339C730F4C2568E604354325605A
:106CC0000468E568B6123543E5600568AE680124DE
:106CD0002643AE6005682E6926432E610568A961CA
:106CE00001684A61006801690422114301619C73D3
:106CF000002070BD00040140704700000448416B53
:106D0000012211434163816B020411438163704787
:106D100000100240C106C90E0120884001490860E8
:106D20007047000080E100E0C106C90E01208840E4
:106D3000014908607047000000E100E010B501F073
:106D400099FA10BD02494A6882434A6070470000C0
:106D500000700040024801688215114301607047CD
:106D60000070004002494A6802434A6070470000D0
:106D70000070004005480168022211430160044888
:106D8000016904221143016130BF70470070004067
:106D900000ED00E00A4B1A689208920002431A6064
:106DA00008480369042213430361012906D040BF48
:106DB00020BF20BF016991430161704730BFF9E7EF
:106DC0000070004000ED00E0F8B504460078544D36
:106DD000800672D5524E0027403EB06BC00004D4EE
:106DE000B06BA9050843B06301274E480168C90587
:106DF00011D40168821511430160FFF7ADFD0090C9
:106E000005E0FFF7A9FD0099401A642837D84548E6
:106E10000068C005F5D532680321090560680A409D
:106E20000140914208D08103890F032904D13168C0
:106E3000890301D50120F8BD2A69032109040A400C
:106E400022D0084090421FD0207880061CD52869A7
:106E50002A6988430121C9040A432A612A698A43AD
:106E60002A612861C0050FD5FFF776FD009008E084
:106E7000FFF772FD0099411A2B48814201D9032086
:106E8000F8BD28698005F3D561688803800F032861
:106E900005D132680005824301400A433260286907
:106EA000032261681204114008432861002F04D0B6
:106EB000B16B012000078143B1632078C00705D082
:106EC000E868A168800880000843E86020788007AF
:106ED00005D5E8680C218843E1680843E86020781C
:106EE000400706D5E86803218902884321690843E1
:106EF000E8602078000706D5E86803210903884385
:106F000061690843E8602078000606D5E868032137
:106F100089048843A1690843E8600020F8BD0000A7
:106F2000401002400070004088130000F8B50E4683
:106F300005007DD053480068C007C00FB0420AD298
:106F40005048016849084900314301600068C007A2
:106F5000C00FB04271D128784B4C800705D5E0684E
:106F6000F0218843A9680843E0602878C00752D020
:106F70006868022817D0032818D02168012818D083
:106F80008905002959DAE168890889000143E1602F
:106F9000FFF7E2FC69680746022912D003291CD0DA
:106FA000012926D033E021688903EAE721688901B5
:106FB000E7E74907E5E7FFF7CFFCC11B334881420C
:106FC00023D8E0680007800F0228F4D123E0FFF700
:106FD000C3FCC11B2D48814217D8E0680007800F11
:106FE0000328F4D117E0FFF7B7FCC11B2748814203
:106FF0000BD8E0680007800F0128F4D10BE0FFF701
:10700000ABFCC11B2148814201D90320F8BDE068D7
:107010000007800FF3D11B480168C907C90FB142AF
:107020000DD901684908490031430160006800E05A
:1070300003E0C007C00FB04201D00120F8BD28789E
:10704000400706D5E068072109028843E96808433C
:10705000E0602878000707D5E0680721C902884367
:107060002969C9000843E06000F036F8E168084A81
:107070000906090F515CC840064908600020FFF767
:107080008DFCF8BD00200240001002408813000073
:10709000CAA9000804010020044805490068C9681D
:1070A000044A4905490F515CC8407047040100205B
:1070B00000100240E3A90008044805490068C968B7
:1070C000044A8904490F515CC840704704010020FC
:1070D00000100240E3A9000810B5184AD1680C203E
:1070E000084004280BD0082810D00C2810D0506875
:1070F0000004410F0120C003491C884010BD1068E6
:10710000C00601D50E4810BD0E4810BD0E4810BD7A
:1071100088020E4B000F185C0902D368890F491CC6
:10712000DB0301D5084A05E01268D20601D5044AFE
:1071300000E0044A5043FDF7DBFF10BD00100240A1
:1071400000093D000024F40000127A00DAA90008CA
:10715000FEB505007ED0FE4CE7680C20E6680740CF
:107160000120000406402878C00747D0082F05D02A
:107170000C2F0AD101200004864206D1206880032A
:107180003CD568680028E5D038E001206968000433
:10719000814203D121680143216011E005230122CE
:1071A0001B0492049942216802D111432160F1E746
:1071B0008143216021680140009120689043206054
:1071C000686800280DD0FFF7C7FB009005E0FFF7C7
:1071D000C3FB0099401A64287AD820688003F6D54A
:1071E0000CE0FFF7B9FB009005E0FFF7B5FB009955
:1071F000401A6428F0D820688003F6D428788007E5
:1072000055D50923E868042F0DD00C2F01D1002E8D
:1072100009D000283BD02168994301432160FFF742
:107220009BFB064627E02168490701D5002891D03D
:1072300061681F22120291432A69120211436160A0
:107240002168994301432160FFF746FFE168090681
:107250000A0F00E079E1BF49895CC840BE49086077
:107260000020FFF79BFB002872D120E0FFF774FBA2
:10727000801B0228B0D820684007F7D560681F211E
:107280000902884329690902084360600FE0206809
:10729000400840002060FFF75FFB064604E0FFF770
:1072A0005BFB801B022897D820684007F7D428781A
:1072B000C0065FD5002F0CD0A869002849D02068EF
:1072C000FF21013108432060FFF746FB06462DE011
:1072D000C0E02068800502D5A8690028A7D06068B2
:1072E000072149038843296A084360606068297F51
:1072F0000002000A090608436060286A410B012069
:10730000C003491C8840E16809060A0F9149895C5D
:10731000C840914908600020FFF740FB002817D1C2
:1073200028E0FFF719FB801B0228A3D820688005FE
:10733000F7D56068072149038843296A08436060DC
:107340006068297F0002000A09060843606011E0B6
:10735000E1E02168FF20013081432160FFF7FCFA62
:10736000064604E0FFF7F8FA801B022872D820686E
:107370008005F7D42878794E000724D5686900285D
:10738000306910D0012108433061FFF7E5FA009021
:1073900005E0FFF7E1FA0099401A02285AD830694F
:1073A0008007F6D50FE0400840003061FFF7D4FABF
:1073B000009005E0FFF7D0FA0099401A022849D85A
:1073C00030698007F6D42878400765D50020029000
:1073D000A06BC00006D4A06B012109070843A0637D
:1073E000012002905E480168C90511D40168821528
:1073F00011430160FFF7B0FA009005E0FFF7ACFA27
:107400000099401A642825D855480068C005F5D56C
:10741000FF20AA680130824203D131690143316102
:1074200011E001218902002A07D005231B029A429C
:1074300003D132690A433261EFE732698243326134
:10744000306988433061A86800280FD0FFF784FABC
:10745000009007E05EE0FFF77FFA0099411A41488B
:10746000814257D830698005F5D50DE0FFF774FAF1
:10747000009006E0FFF770FA0099411A39488142FE
:1074800048D830698005F5D40298002804D0A06B54
:10749000012109078843A063686A002864D00C2F83
:1074A0003ED0012636060228206805D0B043206071
:1074B000FFF752FA05462FE0B0432060FFF74CFA81
:1074C000074604E0FFF748FAC01B022822D82068CC
:1074D0008001F7D4E96AA86AE2680843296BFD23B2
:1074E0001B049A4311430843E06020683043206046
:1074F000FFF732FA054604E0FFF72EFA401B022898
:1075000008D820688001F7D52EE0FFF725FA401B48
:10751000022801D90320FEBD20688001F5D423E0B4
:107520000128F8D0E06801210904AA6A01409142CB
:107530000BD10F218904EA6A0140914205D1032150
:1075400089050840296B88420ED00120FEBD00004D
:1075500000100240CAA900080401002040100240A7
:1075600000700040881300000020EFE770B50400B1
:1075700007D0002625464035A662687C002802D048
:1075800005E0012070BD2E74204600F02FF8022087
:10759000687420680168402291430160A1686068B6
:1075A00022690843E16811430843616901220843E5
:1075B000A169520211400843E1690843216A084366
:1075C000A16A084321680860A0690421000C0840F2
:1075D000616A0843216848602068C169920091434C
:1075E000C161666501206874002070BD10B586B069
:1075F000044614216846FDF7DAFD104920688842E8
:1076000019D10F48416B821411434163C16A0122B1
:107610001143C162C06A002110400590E020009033
:1076200002200190032003900291049105206946F5
:107630000007FFF7C5F806B010BD0000003001409C
:1076400000100240094910B5401E884201D90120AE
:1076500010BD074C60610321081F00F00BFE0020E5
:10766000A06107202061002010BD0000FFFFFF0087
:1076700000E000E070477047F8B502680446D06942
:107680001168936805072D0F5BD0DD07ED0FFF260E
:1076900021360E402E4367D0C60706D0CE0504D54E
:1076A00001261662E26F3243E26787070222042650
:1076B000002F06DADF0704D027683A62E76F374306
:1076C000E767470706D5DB0704D023681E62E36F30
:1076D0001343E367020709D520220A402A4305D055
:1076E000236808221A62E36F1343E367E26F002AFC
:1076F0002FD0800606D5880604D5216E002901D03A
:1077000020468847E06F21688968490601D4000750
:1077100024D5204601F020FF20688168490619D54C
:107720008168402291438160E06E002812D0204998
:107730008163E06EFEF7AAFE00280AD0E06E816B3E
:1077400006E0850610D58D060ED5216E1CE020467C
:107750008847F8BD2046FFF78EFFF8BD2046FFF7AB
:107760008AFF0020E067F8BDC50208D55B0206D598
:107770000120000510622046FFF77CFFF8BD0306DC
:1077800005D50B0603D5616E0029E0D1F8BD400692
:10779000FCD54806FAD51368204640218B43136078
:1077A000202161670021616600F069F9F8BD0000E1
:1077B000B594000810B5040003D0606F002802D013
:1077C00007E0012010BD002170200155204600F087
:1077D00027F8242060672068016849084900016093
:1077E000204601F003FF0128ECD0606A002802D097
:1077F000204601F041FD206841680922D2029143F0
:107800004160206881682A22914381602068016874
:10781000012211430160204601F094FD10BD0000DB
:10782000F0B587B0064614216846FDF7C0FC2C4928
:107830003068884251D12B48416B01229203114399
:107840004163C16A01221143C162C06A0025104030
:1078500005900320400200900220032701A9A1C146
:1078600004200490052069460007FEF7A9FF1F4C7D
:107870001D48A560E56081C48027E560A7602020E1
:10788000256160610002A0611848083CFEF778FE9F
:10789000002801D0FEF772F9F466A662144C124873
:1078A0002146143820600320606010200831A1C1F7
:1078B0006561A561E56120462562FEF761FE00284D
:1078C00001D0FEF75BF9B466002201211B20A662FD
:1078D000FFF734FA1B20FFF727FA07B0F0BD0000CE
:1078E000003801400010024030000240A81500207E
:1078F000F0150020F8B50446806F20284DD10029EE
:107900000BD0002A09D00123A0681B03984206D19E
:107910002069002803D1C80701D00120F8BD254601
:107920006035287C012838D00120287458206165F2
:1079300002530026E6672220A067E06E002819D0D7
:107940001749C162E16E17480863E16E1648486343
:10795000E06E13468663676D21683A462431E06E17
:10796000FEF756FE002805D01020E0672E74202078
:107970006067D2E72E7420680168FF22013211434C
:10798000016020688168012211438160206881685C
:107990004022114381600020F8BD0220F8BD0000A4
:1079A000119500084F950008C9940008704770476A
:1079B000FFB50446406F83B017460D4620285CD1C2
:1079C000002D0AD0002F08D0A168C001814207D144
:1079D0002069002804D1E80702D0012007B0F0BDDB
:1079E000204660300290007C012846D00298012198
:1079F00001740020E06721206067FEF7ADFF264696
:107A000040360190378277820120A16800038142CD
:107A100002D12069002802D02F46002511E000275E
:107A20000FE000228021204601F0F4FE002815D14D
:107A3000002F15D02168387888627F1C708A401E1C
:107A40007082708A019B002806980090E9D100227C
:107A50004021204601F0DEFE002808D00320BDE7CB
:107A600028882168C005C00D8862AD1CE6E720208B
:107A70006067029900200874B0E70220AEE7704703
:107A800001490248C160FDE70400FA0500ED00E08D
:107A900010B505242407002204212046FEF755FFD7
:107AA000002208212046FEF750FF0A2002F0B1F91B
:107AB000012204212046FEF748FF0A2002F0A9F91E
:107AC000002204212046FEF740FF10BD10B505241A
:107AD0002407002204212046FEF737FF0122082157
:107AE0002046FEF732FF0A2002F093F9012204211A
:107AF0002046FEF72AFF0A2002F08BF9002204211B
:107B00002046FEF722FF10BDF8B5002405260746E3
:107B100025463607002204213046FEF716FF0A20CC
:107B200002F077F9012204213046FEF70EFF6006CD
:107B3000040E08213046FEF7FFFE002801D0641C29
:107B4000E4B2052002F065F96D1CEDB2082DE1D319
:107B5000002F03D0FFF79CFF2046F8BDFFF7B6FFCC
:107B6000FAE770B50526054636070022042130469F
:107B7000FEF7EBFE0024E80901D0012200E000221C
:107B800008213046FEF7E1FE6806050E0A2002F0E5
:107B900040F9012204213046FEF7D7FE0A2002F008
:107BA00038F9002204213046FEF7CFFE0A2002F009
:107BB00030F9641CE4B2082CDDD370BD10B5052487
:107BC0002407012208212046FEF7BFFE01220421DE
:107BD0002046FEF7BAFE002208212046FEF7B5FE39
:107BE0000A2002F016F9002204212046FEF7ADFE1D
:107BF00010BD10B505242407002204212046FEF7FD
:107C0000A4FE002208212046FEF79FFE0A2002F073
:107C100000F9012204212046FEF797FE01220821E7
:107C20002046FEF792FE0A2002F0F3F810BD70B570
:107C300005252D070024012208212846FEF785FE90
:107C4000062002F0E6F8012204212846FEF77DFE18
:107C5000062002F0DEF807E0641CE4B2FA2C03D937
:107C6000FFF7C7FF012070BD08212846FEF764FE1C
:107C70000028F1D1002204212846FEF766FE0020EC
:107C800070BD0000F8B501F08DFB01F0C7FB4C485A
:107C90000068C0694B4E4C4F800700D5FE60FEF770
:107CA0005DF84A4C024660884949002803D0401ECE
:107CB000608001200870087801218902454D002864
:107CC0001CD0012804D0022804D0032806D115E0D6
:107CD000212A13D200222846FEF737FE0121C902CD
:107CE0003C48FEF729FE3C490025002828D03B48A7
:107CF00005600846C079002802D006E00122EAE7C4
:107D000035490120C87101F0C9FD33480078632866
:107D100006D9002208212F48FEF717FE012205E0B0
:107D2000012208212B48FEF710FE00220121052028
:107D3000C9030007FEF709FEA08C012803D01CE050
:107D4000CD710022EDE726486946088072B6802191
:107D50002448FDF72BFF002804D002226946214861
:107D6000FDF7C8FF62B620A001F036FEA58402F040
:107D7000ADFD642002F046F8FE60608C012809D158
:107D8000124865844038058002F0A0FD642002F0AE
:107D900039F8FE60208C012806D1258402F096FD7A
:107DA000642002F02FF8FE600848134A403801882A
:107DB000914202D1C088002800D1FE60F8BD0000C9
:107DC000281500200400FA0500ED00E0780D0020E1
:107DD0005B00002000040050C4000020FC000020D4
:107DE000AAAA0000384A0008BDF8C8EBC9FDBCB615
:107DF000C4A3CABD0D0A0000AA55000008B537216A
:107E0000202000F06EF80321212000F06AF84021C4
:107E1000222000F066F80821232000F062F8AA2151
:107E2000302000F05EF80A4802210187322000F07D
:107E300058F80121332000F054F85F21202000F091
:107E400050F8684600F006F80A2001F0E2FF08BD8D
:107E5000380D002010B501460F2000F021F8002851
:107E600000D0012010BD10B50446FFF7A7FE322058
:107E7000FFF777FEFFF7DBFEE0B2FFF772FEFFF7DA
:107E8000D6FEFFF79BFE3320FFF76BFEFFF7CFFE1A
:107E90000020FFF739FE0446FFF7ABFE204610BD79
:107EA00010B50C46FFF7DFFF2070012010BD70B544
:107EB0000D460446FFF782FE3220FFF752FEFFF721
:107EC000B6FEE0B2FFF74DFEFFF7B1FE2846FFF722
:107ED00048FEFFF7ACFEFFF78CFE0A2001F099FF89
:107EE00070BD10B5FFF7E3FF012010BD10B50248CB
:107EF000FEF7F8FD10BD0000A0140020FEB50446FA
:107F0000002572B60068394A831804D13849CD6813
:107F1000032189040D4081680191C1680091416984
:107F20008669002B08D132484038836AC7043B4336
:107F30008362836ABB4383620846304348D02B4840
:107F40002368C34205D12A48C3680322920493439D
:107F5000C360002917D02068026901231A43026117
:107F600020684161FEF7F8FC0746FEF7F5FC216842
:107F7000C01B0968090703D47D21C9008842F4D9D0
:107F8000216808204860002E17D02068016901226E
:107F90001143016120688661FEF7DEFC7D270646FD
:107FA000FF00FEF7D9FC2168801B0968C90601D4CF
:107FB000B842F6D92168102048600C482168C142B7
:107FC00006D10B48C1680322920491432943C16042
:107FD00020680169490849000161216801988860A9
:107FE00021680098C86062B6FEBD00000084FFBF33
:107FF000401002401CB5002116480091144A01911E
:108000000260C1631205426081600722826301221F
:1080100002610246C16020321170FF235170C233E9
:108020004362816211730163816104224163426191
:10803000C161FEF791F808480090801301906946ED
:108040000448FEF739F800210248FDF7DFFF1CBDA8
:1080500000240140441400200200000408B5084830
:10806000016B012211430163006B0121104000905C
:1080700000220A20FEF762FE0A20FEF755FE08BD28
:1080800000100240F0B587B014216846FDF78FF864
:108090004C48C26A04210A43C262C26A0A4005927D
:1080A000C16A80273943C162C16A39400591C16AFA
:1080B00001252943C162C16A29400591C16A02268E
:1080C0003143C162C06A2A463040059005201C2118
:1080D0000007FEF73AFC01223B493C48FEF735FC1D
:1080E00000223B493948FEF730FC9121052000224F
:1080F00009020007FEF729FC3648019000240520FC
:108100006946009502940007FEF75AFB0320019090
:1081100005206946009602940007FEF751FB0C20EB
:1081200000901120019003200390052002946946DD
:108130000007FEF745FB10200090052069460396D6
:10814000019502940007FEF73BFB11200190029479
:108150006946009503941D48FEF732FB1E480190C6
:108160006946009602951948FEF72AFB1B480090C5
:1081700002946946019503941448FEF721FBE80236
:108180006A4651C269461148FEF71AFB9120000267
:108190000090052002946946019503940007FEF7BC
:1081A0000FFB69460948009702950194FEF708FB0A
:1081B000002201210520FEF7C1FD0520FEF7B4FDD8
:1081C00007B0F0BD0010024001060000000400509E
:1081D00008300000000011100000211008360000D7
:1081E00010B50F4C0D482060FF2005306060002066
:1081F000A060E06020616061E061012120624902CD
:108200006062A161A0620720E0622046FFF7AEF93C
:108210002068016840221143016010BD0030014018
:10822000D014002000B585B014216846FCF7BFFFCC
:108230000E480D490160E121490241600021816041
:10824000C160016181610C22C16142610162302122
:1082500041620121090381634900C163FFF7AAFA62
:1082600001F016FB05B000BD0038014028150020C4
:10827000704700008307FF22DB0E9A408907090E32
:10828000994000280BDA0007000F083883080848D7
:108290009B001818C36993430B43C361704783085D
:1082A00004489B001B1818689043084318607047E7
:1082B00000ED00E000E400E0BFF34F8F0449034805
:1082C000C860BFF34F8F00BFFDE700000400FA0550
:1082D00000ED00E0F0B58DB00A2002F077F87D20C7
:1082E000C00002F08DF8F94C0026A670E07B0C2847
:1082F00001D30B20E0730122052051020007FEF795
:1083000024FBE670F248E674F24D007828710221F1
:10831000F148FEF711FB002869D00020A179ED4D4E
:1083200049000843617D89000843E871E06AE8700C
:10833000401CE06260792946A8744200B4310846C6
:10834000A138FCF71BFF06206872E448DF4A00787A
:10835000A872207F287328461338917F0175D17F3A
:1083600041756079002240002946153002F018F965
:10837000607900214000153002F024F9022002F05B
:1083800075F80026EE716674E6720120607326733C
:10839000D348FEF787FC60840546E6706079FDF7F8
:1083A0006DF9D04AD04BFDF763F801F0C7FC01230B
:1083B00000229B07FCF7AAFFFDF7A6F90006C10CF7
:1083C000481980B20121C903A084884201D3401A10
:1083D000A084C648A0632079401C2071C048FEF7E5
:1083E00061FC2084BB48C24D4E3005905BE101200A
:1083F00094E7BB48FEF756FC2084BE4E27460AE0B1
:10840000B748FEF74FFC80B23884B98C884202D35B
:108410004919884206D300210F2001F057FF30424E
:108420003863EDD0386B411C20D040047ED58122CA
:10843000D20100210F2002F088F87D20C00001F059
:10844000DFFF002001F091FF0021102001F03EFF2E
:108450004106A048490E00225030B96401F06CFF7B
:108460009C485030417A0729C0D101E0FFF724FF32
:1084700098480222A0495530FCF7A4FE0028B5D147
:1084800002F0F1F87965386502F0DAF8F965B86557
:10849000F8786946401CF8708E484D3002790A70B1
:1084A000407948700888F98B88427CD10598934EB2
:1084B000008A3080874885494C30808A48838848C4
:1084C000FEF7F0FB3884788B8D49FF30C33080B2E3
:1084D000788388420CD9494240187883308888498B
:1084E000401C80B20B313080884201D300203080A4
:1084F0000598764A81899186C089D0867A6BBA635D
:10850000744A5032D27C13071B0F032B00D0FB742C
:1085100012093A7500233B710123FB726B4B002A51
:108520001987588715D00222734900E0AFE06948E7
:108530005530FCF747FE00280BD1012065497874BF
:10854000C871B86C64311638C2B2BA746D48FCF7A1
:1085500015FE012038735F495C48042251314430D4
:10856000FCF70CFE5B48FB6D1630BA6D02F050F85C
:1085700030887D21C9007A8B41438918F9630791BE
:1085800061490A88D1B23974491E8A4201D1012158
:108590003973F88416203C46385EFDF75BF800918D
:1085A0000490208C00E016E0FDF768F8574A584B1D
:1085B000FCF75EFF06460F460798FDF74BF83B4673
:1085C0003246FCF747FF009B049AFCF79FFEFDF73D
:1085D00077F8206467E0FDF7A9FB064649480321C8
:1085E0000C3881550598394982898A86C089C886A0
:1085F000444AB0009C3A796B11503649FB6D4018E3
:108600001A30BA6D02F004F87879761C86424AD1A5
:1086100001F07AFDFF22A06D5204E16D0023801865
:1086200059410906050A0D4368084000010E000281
:10863000616620662748636D0A30226D01F0E8FF0D
:108640002448636E1230226E01F0E2FF21480821B7
:1086500041726079002280001E491C3001F0A0FFA9
:108660006079002180001C3001F0ACFF284601F049
:10867000A6FE012001F0FAFE0006000E60721AD17B
:1086800000210F2001F022FE0006F9D513E032464A
:1086900000210F2001F059FFF8787979884202D043
:1086A000002001F062FE218CA08C814200D2A0E665
:1086B00040198142FBD80F4A00210F2001F045FFED
:1086C0000021E17363790846049344E048000020E8
:1086D000C4000020AC11002000040050D400002091
:1086E000A0140020B81E85EB51B8CE3FA086010033
:1086F000983A000000D02724E4000020F800002071
:10870000E70300002C130020DA000020F853E3A553
:108710009B843E40614D2A5C002A1AD0E67B8D0086
:10872000761CE6735D4EAC46303E72515B4D4600A2
:10873000C03D4F00AE5B1835EE5386001835574FDD
:10874000AE596546603F7E51491C544D521EC9B218
:108750002A54401CC0B29842DCD3E078032801D2EE
:10876000E07BE0734E490022C87B8873401E33E0F3
:1087700000212DE0494C8B00603C1E19B446E558A1
:108780007668B54222DD0695444D4C00A83D2F5B2E
:108790007835BE469700ED590595404D7746603DCA
:1087A000EE50483D65193D4E0B956D88A83E3553FA
:1087B000344678341E19394D7468303DEC506346A8
:1087C000069D5D600B9D6F80059D7560491CC9B25B
:1087D0008142CFDB521CD2B28242C9DB2F486038C3
:1087E00002682F48816B32398A421CDA2B493039B2
:1087F0000968002917D0C1790246491CC9B2C17164
:10880000032905D92549A8390988D1830221017096
:108810000179032901D901210170204C002103783D
:10882000C03C049A09E00021C171F1E74D00655B8D
:10883000002D00D10223491CC9B29142F6D3037026
:10884000164B0021174C903B8A00491CC9B29C5022
:108850000C29F9D3407C002806D010490C310B7844
:1088600048788A78022B0DD00F4A00210F2001F0A2
:108870006CFE01210520002249020007FEF765F881
:108880000DB0F0BD094BC91C1818FCF777FC02F0BD
:108890001DF8642001F0B6FAE8E50000201300207E
:1088A00048000020FFFF010080D02724380D002061
:1088B00070470000F0B58DB0B54801900020C0436E
:1088C0000A9000260A2001F081FD7D20C00001F001
:1088D00097FD0020AF4C0546A070AF4FAF480B90FE
:1088E000AE480022C23885730146142001F058FEBC
:1088F0000021142001F066FE022001F0B7FD0021E6
:108900000F2001F0E3FC38422063F8D0206B411CBB
:1089100018D040047ED58122D20100210F2001F021
:1089200014FE0021102001F0D1FC41069B48490EA5
:108930000022801C01F000FD9848801C417A022929
:1089400002D005E1FFF7B8FC944802229449C01D0B
:10895000FCF738FC0028F4D101F085FE6165206544
:1089600001F06EFEE165A065002E23D10B988D49C4
:10897000008A088089488749801E808A48830126AA
:108980008948FEF78FF92084608B8849FF30C33017
:1089900080B2608388420DD9494240188149608382
:1089A0000888824A401C80B20B320880904201D372
:1089B000002008800B9968468A890280C989418015
:1089C00076490422C91C0846A238FCF7D7FBFF22CF
:1089D000A16D5204E06D0023891858410006090A70
:1089E00001430846029101F0EAFC02994808400060
:1089F000010E0002616620666848636D9638226D3C
:108A000001F006FE6548E36D9238A26D01F000FEAC
:108A1000624800E09EE08E38636E226E01F0F8FD41
:108A20005E490022A0393C2001F0BAFD00213C2023
:108A300001F0C8FD012001F019FD6072A07801214C
:108A4000401CA0700520C9030007FDF783F95548B5
:108A50007D220088D200014602905043628B0A3981
:108A60008018E0630C90524800782074049008B29B
:108A70002085002803DA7D21C900401820854D4853
:108A8000302100884843FCF7DEFD05902820205E59
:108A9000FCF7CEFD0599FCF7FBFB7F21C905FCF730
:108AA0009EFBFCF7F9FD424980B208800499491EFB
:108AB000884201D1012020730298E0841620205EB4
:108AC000FCF7C8FD05910690208CFCF7D7FD3A4ACB
:108AD0003A4BFCF7CDFC079104900C98FCF7BAFDDB
:108AE000079B049AFCF7B6FC059B069AFCF70EFC64
:108AF000FCF7E6FD2064A08B00F0AAFA009901982B
:108B000081420DDA00290BD024490422C91C0AA88D
:108B1000FCF734FB022020700520A0720098019021
:108B2000607A002805D100210F2001F0CFFB00065C
:108B3000F9D5802200210F2001F007FD00206D1CD7
:108B4000EDB26070032D00D2CAE6002E08D01AE004
:108B50000120F4E71A4A00210F2001F0F6FCF7E7A4
:108B6000A08B1849401E0004000CA08302D00A8884
:108B7000904201D90888A0831349A08B0988401E20
:108B80004843124908800A98E0830DB0F0BD000008
:108B90003F420F004800002000D02724FA11002097
:108BA000E4000020F8000020A0140020E7030000EB
:108BB000DA000020DE000020F853E3A59B843E404D
:108BC00000902724D0000020CE000020CC00002000
:108BD000F8B52F492D48086001F018FE2E4D2D489C
:108BE0006880E888002801D16420E8802B4801785B
:108BF0003C2901D93C210170E98E0170284CE88F95
:108C00006071A88FA071A87AE070AE8805212662F5
:108C10006181EF883846FCF76BFAA0810146304647
:108C2000FCF766FA8800081886B27D20C00026810D
:108C30007043FCF723FD1B4A1B4BFCF781FCFCF740
:108C400063FDE0817D2066823946C000FCF750FA62
:108C500020820146C820FCF74BFA60830120E082A5
:108C6000FDF77CF8A082E28910491148FEF71EF852
:108C700010A0216A00F0B0FEE98812A000F0ACFE5E
:108C8000298915A000F0A8FEF8BD0000C9980008C9
:108C90004400002005020000380D002000000020E4
:108CA000C4000020F853E3A59B843E40FF7F0000F2
:108CB000A0140020B1EAC7A949443A202564202E17
:108CC0000D0A0000CDA8D1B6BCE4B8F43A20256462
:108CD000206D732E0D0A0000B5A5B4CECDA8D1B677
:108CE000BBF9D5BECAFDC1BF3A202564B8F62E0D2A
:108CF0000A000000F0B5924D85B001202880914F08
:108D0000C820914C3880207A401C2072C00706D0C1
:108D1000A08B411EA183022801D2C820A083A08B72
:108D200000F096F90A2001F051FB7D20C00001F00F
:108D300067FB02218548FDF7FFFD002838D00020A1
:108D4000834980000978844E4900084381490978A5
:108D50000843B072102070728048C1887D20C00026
:108D6000FCF7C6F970737E487C490078B0733046D2
:108D70000B308A780270C9784170411C77482030E6
:108D8000027ECA70407E087174482230027E4A71A9
:108D9000407E887100220C39152001F001FC002171
:108DA000152001F00FFC022001F060FB6D4E03E086
:108DB0000120C5E7FEF766FF00210F2001F086FACB
:108DC00030422063F6D0206B411C7DD040047CD51E
:108DD0008122D20100210F2001F0B7FB00211020D9
:108DE00001F074FA41065C48490E00225030A1643B
:108DF00001F0A2FA584E5036707A112865D102223D
:108E00005949701DFCF7DEF900285ED1F01E027989
:108E100069460A7040794870B17A2980C820FCF709
:108E200067F93880307BA083504DB01E008A2880BF
:108E30004549301F808A48834D48FDF733FF80B293
:108E400020840390608B4B49FF30C33080B2608335
:108E500088420CD949424018608328884549401C03
:108E600080B20B312880884201D3002028802D88D1
:108E70007D20C000618B68434018E06302903E484B
:108E8000067828460A3800B226742085002803DABE
:108E90007D21C90040182085388830214843FCF7DF
:108EA000D2FB07462820205EFCF7C2FB3946FCF7C0
:108EB000EFF97F21C905FCF792F9FCF7EDFB2E498C
:108EC00080B20880761E01E037E034E0B04201D184
:108ED00001202073E5841620205EFCF7BBFB0746CB
:108EE00001910398FCF7CAFB244A254BFCF7C0FA12
:108EF00005460E460298FCF7ADFB2A463346FCF7C2
:108F0000A9FA3A46019BFCF701FAFCF7D9FB206469
:108F1000A08B00F09DF868460088E0830E480E495B
:108F20005030807C60714200633108465130FCF75C
:108F300025F90320207005B0F0BDFFF7BDF9000052
:108F4000D4000020DE000020480000200004005073
:108F5000C9000020CA000020AC110020380D0020FC
:108F60000000002000D02724E4000020F8000020AA
:108F7000A0140020E7030000DA000020F853E3A566
:108F80009B843E4070B586B014216846FCF70FF90B
:108F900001250F4EED03002229463046FDF7D5FC92
:108FA0000120002401900294694600950394304604
:108FB000FDF706FC03200190029469460095039496
:108FC0003046FDF7FDFB022000F01CFF06B070BD2F
:108FD0000004005070470000F8B5044600206A46BF
:108FE0001080194D55222A70AA226A700322AA7095
:108FF000661DEE702A716971144A49008918AC71B6
:109000002246E81DFCF7BAF8002007E029186A4656
:109010008978128889186A461180401CB042F5DBB5
:10902000611DA81CFCF706FD014668460180291950
:109030000078C871684640780872214609310248B4
:1090400000F0A2FAF8BD0000E0130020380D002067
:1090500010B51A4CE08A228A6178904201D3801AB6
:10906000E08280B2628B034653435B18238313284C
:1090700002D1424350182083208B30214843642181
:10908000643048430E49E0620968401AA062FCF768
:10909000E1FA0C4A0C4BFCF753FAFCF711FB0B49B5
:1090A0006062884202DD4A4280186062002801DA6C
:1090B0004018606206490968486110BDC40000207C
:1090C00088000020F853E3A59B843E40FF7F00000A
:1090D000A0140020034A1168382389B29943014340
:1090E000116070470030014010B5FDF73BFC10BD2A
:1090F00010B59AB034216846FCF759F814210DA830
:10910000FCF755F81C2112A8FCF751F81B48016820
:109110000324E402A143C21489180160FDF71AFE7A
:1091200017480169A143016106200090FF2001302A
:109130000290012003901020049002200990400426
:109140000B90000100240C900A946846FEF700F88A
:109150000F200D9003200E900F9410940121119474
:109160000DA8FDF7E3FE81201290032080041890E3
:10917000149412A8FDF728FE1AB010BD007000402C
:109180004010024010480168821511430160C16817
:109190000E4A1140C16001680D4A114001608168AA
:1091A00049084900816001680122920491430160ED
:1091B000C168FD2212049143C1600021016106498A
:1091C0000448886070470000001002400C40FF888F
:1091D000F6FFF6FE0050000800ED00E070B501F06B
:1091E00089F8234C234DE06402E001F083F8E06449
:1091F000A842FAD1207801260525F6032D0700287C
:1092000006D001280CD0022817D003282CD129E041
:10921000012231462846FDF798FBFFF76BFD06E07B
:10922000012231462846FDF790FBFFF743FB002261
:1092300031462846FDF789FB16E0A07A0122401E40
:10924000A07231462846FDF780FBFCF7A3FD002203
:1092500031462846FDF779FBA07A002804D1012089
:10926000207001E0FFF736F800F036FF70BD000017
:10927000480000203001CADE10B5818CC90707D034
:1092800001684A6801235B049A43836A1A434A606F
:10929000818C890707D501684A6801231B049A431A
:1092A000C36A1A434A60818C490707D501684A6836
:1092B00001239B049A43036B1A434A60818C09077C
:1092C00007D501684A680123DB039A43436B1A43BD
:1092D0004A60818CC90607D50268916801231B0387
:1092E0009943836B19439160818C890607D5016886
:1092F0008A6801235B039A43C36B1A438A60818C9B
:10930000490612D503685A6801210905046C8A438D
:1093100022435A60026C8A4207D1026851680323D3
:109320005B059943436C19435160818C090607D54D
:1093300001684A680123DB04806C9A4302434A6057
:1093400010BD0000F8B500260446C667FDF704FB13
:10935000054620680068124F000709D501212B46F9
:10936000002249052046009700F054FA00280DD14C
:109370002068006840070BD501212B460022890593
:109380002046009700F046FA002801D00320F8BDDF
:1093900020206067A067603426740020F8BD0000BC
:1093A000FFFFFF01F8B5184CC826E078002829D146
:1093B0006079002826D101206071144D686B002768
:1093C00000281ED0686BC821081A15E01048E16813
:1093D000405C616988470F480A21008848430E496C
:1093E0000880E068401CE060E068C82800DBE760B7
:1093F000696BC820401A761EE168814201D0002EB8
:10940000E4DC6771F8BD000030000020000002407D
:10941000700C0020D4000020E000002070B5224C29
:10942000E07800283FD1207900283CD1012020712C
:109430001E4EF16900250906002933DA21566257CC
:1094400091420AD1F06940062CD5A079002829D094
:10945000A5712089401C208124E0A179002903D135
:10946000A0710A2000F0D5FC00202056CC214843F2
:109470000F494218206912181279B262401C00226A
:109480002061A256CC235A43895881420ADC2561C7
:109490002078401C207020780E2800D12570A078FC
:1094A000401CA070257170BD3000002000380140C4
:1094B0004801002010B5806A0022014640314A83ED
:1094C0004A82FEF7D8F810BD70B5846A606FA56F48
:1094D0002168896800260906002906DA212804D1B6
:1094E00052200653204600F047F820688068400666
:1094F00006D5222D04D15A200653204600F02CF820
:10950000E06F10210843E0672046FEF7B4F870BD15
:1095100010B501460968806A0968890614D40022DA
:109520005A210A5201680A68FF2301339A430A60EC
:1095300001688A68520852008A6001688A6840237C
:109540009A438A6020218167FEF730FA10BD10B57A
:10955000806AFEF72CFA10BD01680A68FF232133E8
:109560009A430A6001688A68520852008A60202182
:10957000816700210166704701680A68C0239A4329
:109580000A6020214167704770B5164CE278002AC6
:109590000CD12279002A09D10122E2700025C829C4
:1095A00003DC0222A256002A01DCE57070BD012313
:1095B000E356CC2253430C4AD1500123E356CC2628
:1095C00073439B180A460146181DFBF7D7FD6078C8
:1095D000401C607060780E2800D16570A078401E35
:1095E000A070E2E73000002048010020F8B50446F2
:1095F0002669A268E76932436669102000253E4368
:109600002368324378491E68784F3E4016431E60F7
:1096100023685A6803263603B243E66832435A6029
:109620002368A2698B4201D0266A32439E680B27C9
:109630003F02BE4316439E606D4E23686D4AB3429F
:109640000CD1D2689207920F06D0012A38D0022A94
:1096500034D0032A20D11EE001201DE0664EB34223
:109660000AD1D2680C26324026D0042A28D0082AF3
:1096700024D00C2A10D10EE08B420DD1D6680322E3
:109680009202164018D001229202B61A18D0B61AC9
:1096900014D0964200D10820564A0126403A574F2E
:1096A000F6038B4236D100280CD002280DD00428B6
:1096B00012D008281FD11CE00020EDE70220EBE7C4
:1096C0000420E9E7FDF7E8FC08E01068C00601D5D2
:1096D000384605E04A4803E0FDF7FEFC002873D059
:1096E000626851005118814205D81103814202D3AA
:1096F00003E03046F4E7012566E0010E060250085B
:10970000002330185941FBF709FD03210902411AD2
:109710003C4A55E0E169B14232D1030000F083F9DF
:1097200009070A0D06250606062B0600E3E7FDF7E6
:10973000B3FC1CE0FDF7C0FC19E010686168C006CE
:1097400002D54808304A01E0304A48088018FBF743
:10975000CFFC80B201462E4A10399142CBD8511C21
:1097600001400007400F08432CE0FDF7B5FC61689D
:1097700040004A08EAE76168012248081204E5E768
:10978000030000F050F909070A0D06260606062C0C
:109790000600B0E7FDF780FC1DE0FDF78DFC1AE048
:1097A00010686168C00602D54808C01902E0144874
:1097B0004A081018FBF79CFC80B20146144A103985
:1097C000914298D82168C8600020206660662846CB
:1097D000F8BDFDF781FC61684A088018EAE7616816
:1097E00048088019E6E7000000480040F369FFEFF1
:1097F00000380140401002400044004000093D0094
:109800000024F400FFFC0F0000127A000048E80179
:10981000EFFF0000FFB581B017460E4604460A9DD3
:1098200009E0681C07D0FDF797F80499401AA84290
:109830000CD8002D0AD02068C1693046884318D062
:109840000020B842EDD0002005B0F0BD20680168CE
:10985000FF22A132914301602068816849084900D4
:10986000816020206067A06700206034207403209E
:10987000EAE70120E5E7000010B504491020096877
:1098800008620248FDF7F8FE10BD00002815002010
:1098900001490D20887070473000002010B507483E
:1098A0000A22018A51438183FEF7D8FBFEF7BAFCF6
:1098B000C82203490348FEF71DF810BDC40000206C
:1098C000700C002028150020F8B53E4C00232178AC
:1098D0003D4A1D46082910D0072947D0062950D0F7
:1098E000052952D0042953D0032954D0002956D039
:1098F000012958D002295AD05BE0A17800264A1FDE
:1099000004E0314FBF5DFB189BB2761C9642F8DB3A
:10991000667927799A195118E3786278C9188918F5
:10992000C9194018C0430006000E1AD1012E14D0E8
:10993000022E16D125482449C018FBF71FFC00F061
:10994000C5FF642000F05EFABFF34F8F2149204825
:10995000C860BFF34F8F00BFFDE759081046FFF7FF
:109960003BFB2570E570A570A571F8BDA179505439
:10997000491CC8B2A071A178491F8842F5D10820BE
:1099800001E0607007202070F8BDE0700620FAE763
:1099900060710520F7E7A070E5700420F3E7552813
:1099A00007D10120EFE7AA2803D10220EBE7032823
:1099B00003D02570E570A570F8BD032020702071DC
:1099C000F8BD0000BB0000207C130020380D0020F3
:1099D0000400FA0500ED00E00FB410B503A9044B34
:1099E000044A029800F002F910BC08BC04B0184701
:1099F00029A60008080100202021020C01D0102116
:109A00001046020A01D010460839020901D010465A
:109A1000091F820801D01046891E420801D0881E05
:109A20007047081A704730B47446641E2578641C69
:109A3000AB4200D21D46635D5B00E31830BC1847A3
:109A400002E008C8121F08C1002AFAD17047704707
:109A5000002001E001C1121F002AFBD1704708B5A8
:109A60000021684601706B46012202212C2000F083
:109A70007BFD0221684601706B4601222C2000F01C
:109A800073FD08BD38B504466D20694608706B4605
:109A9000012207492E2000F067FD0649002C01D065
:109AA000054A00E0054A2E2000F044FD38BD0000C4
:109AB0000608000006180000070600000716000050
:109AC00038B504466B4602220021362000F018FC0F
:109AD000B3212300FFF7A7FF0E0F08153A3A3A3AD1
:109AE0001C273A3A2F34483A0021684601704078E2
:109AF0004108490014E06946087880088000401C4D
:109B000004E06946087880088000801C08701DE029
:109B1000684602780A40483202704178802001434A
:109B20006846417012E0684602780A400270407848
:109B30004106490EF4E7694648780221084303E0EC
:109B400069464878FD210840694648706B46012205
:109B50000021362000F008FD012200AB114636201E
:109B6000013300F001FD38BD69460878CF21084077
:109B700069462030CAE708B50321684641700121D3
:109B800001706B4602220021362000F0EDFC01221C
:109B9000D20306212D2000F0CDFC012000F032F987
:109BA0000120FFF78DFF08BD08B5020A69464A701B
:109BB00008706B46022204212D2000F0D5FC032002
:109BC000694608706B46012206212D2000F0CCFC6E
:109BD0000020694608706B46012206212D2000F006
:109BE000C3FC0A212D2000F071FB08BDFFB58DB02C
:109BF0000446002506E025280AD0109A0F999047C0
:109C0000641C6D1C20780028F5D1284611B0F0BDE9
:109C100000270121484A009700E00743641C23788D
:109C20000846203B98401042F7D120782E2817D1C3
:109C3000042007436078641C2A280CD10E98641C09
:109C400002C800910E900BE000990A22514330396E
:109C50004018641C00902078014630390929F3D956
:109C600020780028D1D0642808D0692806D075282B
:109C70001ED0109A0F9990476D1C5BE00A200E9938
:109C8000019001C90E91002802DA40422D2102E024
:109C9000390504D52B216A461172012103E0F90729
:109CA00004D02021F7E70BAE0B910DE00021FAE77D
:109CB0000A200E99019001C90E91F7E70199FBF76F
:109CC00017FA3031761E31700028F7D103A8801BB7
:109CD00020300190780701D5009801E00120009024
:109CE0000199884201DD401A00E000200027009021
:109CF00006E002A8109AC05D0F9990476D1C7F1C6A
:109D00000B988742F5DB04E0109A30200F999047BA
:109D10006D1C0099481E00900029F5DC05E03078A4
:109D2000109A761C0F9990476D1C0199481E01905E
:109D30000029F4DC641C65E709280100F8B54A0035
:109D40002B4B520DD6182B4A0C460546142E2BDAF7
:109D5000002E12DA284BFBF7D9FA00221346FBF744
:109D6000FFFD40D2002C03DA0124E40700253AE08D
:109D70002046284337D0214C14E0214F0B46F740B2
:109D80003B402B4331D01C4BFBF7C0FA002213465B
:109D9000FBF7E6FD27D2002C03DD01200005F04093
:109DA0000419BC4300251EE0332E1EDC3346002779
:109DB000143BFF43DF40384217D00F4BFBF750FBFB
:109DC00000221346FBF7CCFD0DD2002C0ADD142E29
:109DD0000CD03420811B012088404019A84200D2B9
:109DE000641C0546BD4321462846F8BD641CF9E7BE
:109DF00001FCFFFF9C7500883CE4377E0000F03FCB
:109E0000FFFF0F007D2110B5C900484300F001F8A5
:109E100010BD002140E000BF00BF00BF00BF00BF79
:109E200000BF00BF00BF00BF00BF00BF00BF00BF3A
:109E300000BF00BF00BF00BF00BF00BF00BF00BF2A
:109E400000BF00BF00BF00BF00BF00BF00BF00BF1A
:109E500000BF00BF00BF00BF00BF00BF00BF00BF0A
:109E600000BF00BF00BF00BF00BF00BF00BF00BFFA
:109E700000BF00BF00BF00BF00BF00BF00BF00BFEA
:109E800000BF00BF00BF00BF00BF00BF00BF00BFDA
:109E900000BF00BF00BF491C8142BCD37047000017
:109EA000FEB504460020019000906079734940009F
:109EB0000E5A61782578491E7148CFB20163042D8E
:109EC00077D0072D75D000210291217801736C495C
:109ED000E379012292058969002B6CD0914381615D
:109EE0006748217A4173217A82698907890B0A437D
:109EF00082610021042000F028FB324661492E20B7
:109F000000F018FB3846FFF7BDFD5F4E0522705D7F
:109F1000810040185D49431807212B2000F024FBE5
:109F20005B49029801220B180B21282000F01CFB32
:109F3000705D584980000A580C21282000F005FB6C
:109F4000E079554980004018A1794900425A022120
:109F5000272000F0EFFA51487E00825B0421272081
:109F600000F0E8FAE079002829D0A07804282CD065
:109F700028206946087220220621272000F0DAFAFC
:109F800002AB01222621272000F0EEFA44493801D5
:109F90004018E178890042580821272000F0D5FABE
:109FA000A17A601C627A0902114313D016E000E026
:109FB00001E0012188E71143F608816190E76422FE
:109FC0000621272000F0B6FAE0E710206946087263
:109FD0000246D1E733490172090A4172417A007A97
:109FE0000A0202432021272000F0A4FA2E4F0C2160
:109FF00023203A6800F0A9FAF0198288042123206E
:10A0000000F098FAA07900280BD0E07927490122C6
:10A0100043180021212000F0A7FA0320019001201D
:10A0200000902A07120F1001024360780021800778
:10A03000000B0243019800050243009840040243CC
:10A040002079C006400902436079C00602431F2000
:10A0500000F07BFAA07861780123084302040848E5
:10A06000DB030261E179490319430A4302610021DC
:10A07000082000F06AFA0020FEBD000098A9000840
:10A080000C0100200428000040A900080100002065
:10A090001F00002048A9000868A9000874A900084A
:10A0A00078A900084110000060A9000821000020E4
:10A0B00038B50C4607498A8B002102432C2000F05A
:10A0C00039FA684604706B46012206212C2000F004
:10A0D0004BFA38BD0C01002010B5FFF7C0FC10BDD5
:10A0E00010B504460421362000F0F0F80121C90221
:10A0F000002C01D0084300E08843024604213620AA
:10A1000000F023FA10BD000038B540206946087001
:10A1100000210E2000F0DAF80446002211460E203D
:10A1200000F013FA6B46012200210D2000F01CFA0A
:10A13000074A00210F2000F008FA00F0E1F922465A
:10A1400000210E2000F001FA02480021017338BD01
:10A15000F8FF27242C0100207CB505460420694621
:10A1600008704B4C002060752146203120634871F7
:10A170000873A0836063A06300F0BCF8454E2060C4
:10A1800002E000F0B7F82060B042FAD10020FFF7FB
:10A1900097FC41480078242801D9243806E006219C
:10A1A000FAF7A6FF0622101A40010843020601042E
:10A1B0000A4301020A43024300211E2000F0C5F9B0
:10A1C0006B4601220021242000F0CEF91E20FFF76B
:10A1D000EBFC86B2300AA0730420FFF7E5FC000612
:10A1E000000E0DD002206946087101AB0122122138
:10A1F0002D2000F0B9F9A08B012109030843A083A9
:10A2000000F078F820600620FFF7CEFC60600720A1
:10A21000FFF7CAFCA060F006C00E207501D1102027
:10A220002075C0B200F0DCF9E80707D0FFF7A3FC07
:10A23000A08B0121C9020843A0830AE00521362032
:10A2400000F02EF81549084002460521362000F09E
:10A2500071F90120FFF734FC0021042000F036F8EA
:10A26000A0610021262000F031F815218903084360
:10A2700002460021262000F068F90022262136201F
:10A2800000F058F900F036F8206000207CBD000096
:10A290000C0100203001CADE00000020FFFD00009C
:10A2A00038B5094C89B280B26B46022200F028F81A
:10A2B000002806D1684640780102684600780818F0
:10A2C00084B2204638BD0000FFFF000038B50024EE
:10A2D000E44389B280B26B46042200F011F80028F2
:10A2E00006D103216846435C2202D418491EFAD5E0
:10A2F000204638BD10B500210846FFF7E7FF10BD26
:10A3000038B5002909D0402420436C462070C8B2DB
:10A310007F2906D8607002200AE069460870012093
:10A3200006E0802420436C466070C809A0700320BA
:10A33000694600F0A5FA38BD10B5144603460A4632
:10A3400021461120FFF7DCFF10BD10B503460522A2
:10A3500000211520FFF7D4FF10BD10B503460522DC
:10A3600000211720FFF7CCFF10BD38B505460020AF
:10A370006946087000F0C4F8FF2401342246002D1D
:10A3800001D00322120200210D2000F0D3F8002D8D
:10A3900013D06B46012203210F20FFF7B1FF68465F
:10A3A0000078000709D5FFF7AFFE224600210D20F7
:10A3B00000F0C0F80020C04338BD002038BD10B503
:10A3C000024601210A2000F0C0F810BD10B5044675
:10A3D00000211A20FFF77AFF000D22030005120B5F
:10A3E000024300211A2000F0B0F810BD10B502465B
:10A3F00002492E2000F09EF810BD00000418000055
:10A40000F8B505466B46012203210420FFF778FFCB
:10A410000126114C3607002D0DD02A4600210C20B4
:10A4200000F088F8694608781021084369460870EA
:10A43000A069304307E069460878EF210840694683
:10A440000870A069B0430B46A061012203210420DB
:10A4500000F08AF8F8BD00000C01002010B502469B
:10A460000021182000F066F810BD0000F8B507467E
:10A47000002568460570B807204C2E4600280ADAE9
:10A480008020694608706B46012200210D2000F0F3
:10A490006BF801202073F8076946087821D006215F
:10A4A0000843694608706B46012200210D2000F028
:10A4B0005BF803210F20FFF7F3FE8121C90008425A
:10A4C00019D04020694608706B46012200210D20FA
:10A4D00000F04AF80020FFF703FE00252673ED4345
:10A4E00009E002210843694608706B4601220021F9
:10A4F0000D2000F039F82846F8BD00002C0100209E
:10A500001CB56B46012203210F20FFF7F9FE6846B8
:10A5100000784022C1091040C9014000814208D0A2
:10A52000012069460871024601AB03210D2000F0AD
:10A530001BF81CBD08B56B461A70120A5A7089B216
:10A5400080B2022200F010F808BD38B500236C4636
:10A55000E254120A5B1C042BFADB89B280B2234658
:10A56000042200F001F838BD38B58024002909D054
:10A57000C02528436D462870C8B27F2907D8687067
:10A58000022009E0204369460870012004E02043CE
:10A590006870C809A8700320694600F0ADF938BD9D
:10A5A00010B51446012312189B029A4202D90020CA
:10A5B000C04310BD0B46821E21460920FFF7D4FF81
:10A5C000002010BD10B5054A8905126901430A43F0
:10A5D00000210820FFF7B9FF002010BD0C0100206A
:10A5E00038B504466B4601220E212B20FFF788FE6A
:10A5F00068460078E10640094001C90E01436846FB
:10A6000001706B4601220E212B20FFF7ADFF38BDF4
:10A6100010B5002142541C06120A22431B0A491C91
:10A620000429F7DB10BD000013B501231A46694663
:10A630000248FDF7BDF900981CBD00002815002058
:10A640007CB5002425466846FFF77FFE0420694656
:10A65000220E2D02154322020C5C1443401EF7D536
:10A66000204629467CBD7CB5002425466846FFF778
:10A6700074FE04206946220E2D02154322020C5C52
:10A680001443401EF7D5204629467CBDFCF772F9DD
:10A69000FEF72EFDFDF7F6FC37493848002522C0AD
:10A6A00005608561C56136490562C1600838FCF7FF
:10A6B0007FFAFDF7D3FCFDF7B5FDFDF791FDFDF742
:10A6C00099FC052601223607D1033046FCF73DF9F7
:10A6D000FEF77EFAFDF792FBFBF70CFAFBF7DAF9CF
:10A6E0000721B015FFF7E4FC264C0A21208A01223D
:10A6F0004843A083170339463046FCF726F91F4824
:10A70000C82221498830FDF7F5F8204E207900282D
:10A710002FD0FEF7EDFC2571FBF704FC20700F280D
:10A7200009D9012239463046FCF70FF9FEF756FDEC
:10A730000022394609E0012251033046FCF705F9B1
:10A74000FEF74CFD0022012149033046FCF7FDF8DD
:10A75000FDF798FAA08B002801D0401EA0830C487A
:10A76000A18B00780843D1D101210846FCF712FBE8
:10A77000CCE7FDF787FAC9E7007C0040A014002071
:10A78000FFFF0000C4000020700C002000040050F7
:10A790003600002010B586B01748FCF78EF914215A
:10A7A0006846FAF704FD1548009003200190002048
:10A7B0000290052069460007FCF702F86946104838
:10A7C000FBF7FEFF69460F48FBF7FAFF0121084639
:10A7D000FCF7E0FAFF2401342046FCF7B3FA0A49FB
:10A7E00008680422104308602046FCF7BBFAFCF717
:10A7F000C1FA06B010BD0000A0140020FFFF000049
:10A8000000040050000800500070004010B5012204
:10A81000920218491848FBF7E3F9164817490288CD
:10A820008A4225D0018004218180FF21F531C18039
:10A830000A21018100211E224181D243828101220D
:10A84000C2810184018241828182C182018381832C
:10A850001E23C38602230387782343878287C28708
:10A8600002464032118451849184C18300F02EF855
:10A8700010BD0000380D002000FC0008AA550000A3
:10A88000F0B58C4600251026052109078E620E4C76
:10A8900008E067467F5DE760A768FF07FCD0E768D0
:10A8A0001F706D1C8542F4DB0020074606E0E76060
:10A8B000A568ED07FCD0E5681D54401C9042F6D316
:10A8C0008E610020F0BD00000030014070B572B60E
:10A8D0000124074DA40221462846FBF767F900280A
:10A8E00004D0224603492846FBF704FA62B670BD3D
:10A8F00000FC0008380D0020F0B5002510260527C3
:10A900009C463F070B46BE620C4C06E0595DE16079
:10A91000A168C907FCD0E1686D1C8542F6DB002008
:10A9200007E06146095CE160A168C907FCD0E16805
:10A93000401C9042F5D3BE610020F0BD00300140C4
:10A940000000010203040005405C0000A05C04005C
:10A95000C06C0800805C0400E03F1E00E07D1E002B
:10A9600007A9022570889B880A00160001000600CE
:10A970000100020087008D002D001A3152001A33A9
:10A980009A001A351D011A376B003B31BE003B336C
:10A990005E013B3596023B37000099599959EB51BE
:10A9A0008F421E45142E0080EB51F5283333E13AD7
:10A9B000703DE13AC235852BC2353333C235C235DD
:10A9C000AE47E13A5138A330513800000000000092
:10A9D00000000102030406070809030406080C101E
:10A9E0001820300000000001020304000CAA000837
:10A9F000000000200C010000409A000818AB00087D
:10AA00000C01002044190000509A000800070400BF
:10AA1000091E080540082609104008560805400888
:10AA2000261D040008BE1D040008BED8BC40100846
:10AA3000010000000000C84200000000000000000B
:10AA40000000000000000000000000000000000006
:10AA500000000000000000000000000000000000F6
:10AA6000000000000000000000005C120000000078
:10AA700000000000000000000000000000000000D6
:10AA800000000000000000000000000000000000C6
:10AA900000000000000000000000000000000000B6
:10AAA00000000000000000000000000000000000A6
:10AAB000000000000000000000000000020204008E
:10AAC00009090102008100000000000001000000EF
:10AAD0000003000000000000000000000000000073
:10AAE0000000000000000000000000000000000066
:10AAF0000000000000000000000000000000000056
:10AB00000000000000000000000000000000000045
:08AB100000002000000000001D
:04000005080050C1DE
:00000001FF
